:020000040000FA
:06000000F3EF0EF0120008
:06080000F3EF0EF0120000
:06082A0001004C1E00005D
:0808300000020000200000009E
:0808380058EC09F0FB0EDBCFC8
:10084000F3FFDB06F35000090AE0A6EC09F0FA0E0C
:1008500011EC0AF0F3E1151CF1E1010E01D0000EDC
:1008600087EF09F058EC09F03B0EE12402E3E16860
:10087000E652E16E010EDB6A020EDB6AF90EDBCF97
:10088000F6FFFA0EDBCFF7FFFB0EDBCFF8FF080019
:10089000F550DF6EDF5002E1ABEF08F0250EDF5CB4
:1008A00002E09EEF08F0030EDB6A040EDB6A050E21
:1008B000DB6A060EDB6A070EDB6AC0EC08F02D0E61
:1008C000DF5C0CE02B0EDF5C09E0200EDF5C06E055
:1008D000230EDF5C03E0300EDF5C1AE1DF50300AEC
:1008E00014E0130A0FE0030A0AE00B0A05E0060A07
:1008F000E4E1030EDB80E1D7030EDB82DED7030EDB
:10090000DB84DBD7030EDB86D8D7030EDB88D5D795
:100910002A0EDF5C1BE1BCEC08F00AEC09F010E0E9
:10092000030EDB8008680968130EDBCF0DF0140E90
:10093000DBCF0EF070EC0EF0040E06C0DBFF03D030
:10094000130EF3EC08F0C0EC08F00BD0090EDB6AD4
:1009500061EC09F003E0D5EC09F0FAD7090EF3ECED
:1009600008F0030EDBB0DB982E0EDF5C1BE1C0EC61
:1009700008F02A0EDF5C0BE1BCEC08F00AEC09F091
:1009800003E1130E45EC09F0C0EC08F00BD0090EA2
:10099000DB6A61EC09F003E0D5EC09F0FAD7090E47
:1009A00045EC09F0680EDF5C07E1C0EC08F0680E6A
:1009B000DF5C1DE1030E18D0740EDF5C17E07A0EC9
:1009C000DF5C14E0480EDF5C06E0540EDF5C03E001
:1009D0005A0EDF5C02E1020E07D06C0EDF5C03E012
:1009E0006A0EDF5C04E1010E98EC09F0C9DBDF5010
:1009F0006E0A01E17FD31E0A01E192D1200A01E1D2
:100A00008FD13F0A01E149D11A0A01E146D10D0A0D
:100A100001E143D1200A01E140D13A0A01E13DD18F
:100A2000200A01E13AD1260A01E135D10D0A01E19E
:100A300032D11A0A01E1D9D0200A4AE0300A1FE077
:100A4000460A0EE0250A01E083D3D950F90FE96E7A
:100A5000FF0EDA20EA6E010EEE5E000EEE5AEE5A3E
:100A6000A6EC09F0250EE66E95DB03E1151C01E10D
:100A700069D3A2EC09F001E26BD3DB2A69D3080E3B
:100A8000DB6A040EDB50010806E2040EDB046AECAC
:100A900009F0DB508BDB080EDB5009E0030EDB5066
:100AA000010B05E172DB01E04DD3080EDB6A64DB6C
:100AB000EFCFDFFF1AEC0AF003E1151C01E142D38E
:100AC000A2EC09F001E3DB2A60DB01E141D33AD378
:100AD000070EDB5002080FE1E6EC09F0030EADEC67
:100AE00009F00E0EEECFDBFF0F0EEECFDBFF100E88
:100AF000EECFDBFF20D0F70EDBCF17F0F80EDBCF09
:100B000018F0020E175E000E185AF70E17C0DBFF22
:100B1000F80E18C0DBFF17C0E9FF18C0EAFF9DEC14
:100B200009F0166A0E0E14C0DBFF0F0E15C0DBFFB6
:100B3000100E16C0DBFF0E0EDBCFE6FF0F0EDBCF75
:100B4000E6FF100EDBCFE6FF4BEC0EF0E552E55270
:100B5000E552130E07C0DBFF140E08C0DBFF060EC4
:100B6000DB5005E0130EE1EC09F001E26ADB05EC75
:100B70000AF002E2130E37DBC8EC09F006E0040EBF
:100B8000E1EC09F002E2050E2EDB030EDBB005D02E
:100B9000FCDA01E0D7D2080EDB6A090EDB6A0E0E22
:100BA000DBCFF6FF0F0EDBCFF7FF100EDBCFF8FF2A
:100BB0000800F550DF6EDF5014E00BEC0AF011E294
:100BC0001AEC0AF003E1151C01E1BCD2BBDB01E326
:100BD000DB2A090EDB2AD9500E0FE96E000ECBDBA3
:100BE000E7D7D3DA01E1B4D2ADD2C6DA110EEECF37
:100BF000DBFF120EEDCFDBFF110EDBCFE6FF120E97
:100C0000DBCFE6FF3DEC0EF0E552E552130EF3CFDD
:100C1000DBFF140EF4CFDBFF060EDB5004E0130EF7
:100C2000D0DB01E20EDB05EC0AF002E2130EDBDAA8
:100C3000AFDB05E0040EC5DB02E2050ED4DA030EDD
:100C4000DBB005D0A2DA01E07DD2080EDB6A090E26
:100C5000DB6A110EDBCFE9FF120EDBCFEAFFEFCF2D
:100C6000DFFFDF5014E0D7DB12E2E4DB03E1151C09
:100C700001E168D267DB01E3DB2A090EDB2A110EF2
:100C8000DB2ADBCFE9FF120EE8E3DB2AE6D77DDAC9
:100C900001E15ED257D2030EDB8E070EDB0410E1BA
:100CA00095DB040E5ADB0A0EEECFDBFF0B0EEECF08
:100CB000DBFF0C0EEECFDBFF0D0EEECFDBFF6CD0BB
:100CC000070EDB5003082CE1030EDBAE0DD0B2DAC9
:100CD000020E76DAEFCF14F0156A166A176A14AEB0
:100CE00039D01568166835D0F70EDBCF15F0F80E41
:100CF000DBCF16F0020E155E000E165AF70E15C069
:100D0000DBFFF80E16C0DBFF15C0E9FF16C0EAFFD7
:100D1000EFCF14F00A0E14C0DBFF0B0EDB6A38D0E5
:100D2000070EDB50020809E1030EDBAE04D059DBED
:100D300016AE10D00ED055DB0DD0030EDBAE12D0A8
:100D400079DA020E3DDAF9DA166A176A15AE02D0C0
:100D500016681768E2DA0C0E16C0DBFF0D0E17C01E
:100D6000DBFF1AD0F70EDBCF16F0F80EDBCF17F053
:100D7000020E165E000E175AF70E16C0DBFFF80EB5
:100D800017C0DBFF16C0E9FF17C0EAFFD6DAC5DAE5
:100D90000C0EDB6A0D0EDB6A060EDB5005E1010E60
:100DA000F36E050EF3CFDBFF150EDB6A160EDB6A62
:100DB000D950370F146E000EDA20156E390E14C09C
:100DC000DBFF3A0E15C0DBFF380EDB6A080EDB6A6C
:100DD0000A0EAEDADF50780A12E0200A10E0280A84
:100DE0000CE0200A0AE03F0A06E00D0A02E0200AB1
:100DF00008E1020E05D0080E03D0080EDF26100E03
:100E000097DA030EDBBE02D0DB92DB94DB50800B63
:100E100024E08ADAD890030EEB50000A08E6000EB0
:100E2000EE5C000EEE58000EEE58000EEE5815E285
:100E300013DA0B680C680D680E6805EC0EF00A0EEC
:100E400002C0DBFF0B0E03C0DBFF0C0E04C0DBFF98
:100E50000D0E05C0DBFF2D0E08D0030EDBA202D065
:100E60002B0E03D0DBA408D0200EF36E170EF3CFA9
:100E7000DBFF150EDB2A02D0170EDB6A050EDB50F6
:100E800003E1B7D901E189D0340E146E1E0E156E40
:100E9000000E166E070EDBCF17F0186A196A1A6A71
:100EA00017C00BF018C00CF019C00DF01AC00EF0EE
:100EB000D3D99DEC0EF014500224F36E155003208C
:100EC000F46E16500420F86EF4CFF7FFF3CFF6FF60
:100ED0000800090EF5CFDBFF580EDF5C0FE1610E55
:100EE000F36E090E7BD90AE3200E146E090EDBCFD8
:100EF000E7FF1450E75E090EE7CFDBFF070EDBCFFD
:100F000014F0156A166A176A0FDA14C00BF015C0D0
:100F10000CF016C00DF017C00EF0EECF06F0EECFBD
:100F200007F0EECF08F0EFCF09F09DEC0EF009C00E
:100F3000EDFF08C0EDFF07C0EDFF06C0EFFF390E63
:100F4000DBCFE9FFDB063A0EDBCFEAFF01E2DB068F
:100F5000090EDBCFEFFF150EDB2A4BD995E1030E0F
:100F6000DBA61DD06F0EDF5C06E1C1D918E3150EBC
:100F7000DB285BDA14D0780EDF5C09E0580EDF5C0A
:100F800006E0620EDF5C03E0420EDF5C08E1020E69
:100F9000F36E160EF3CFDBFF02D0150EDB6A030EE5
:100FA000DB50100B0EE0040EDBCF14F0050EDB500F
:100FB000D880145406E2060EDB5003E1040EDB5029
:100FC00034DA95D90AE2050EDBCFE7FF150EDB50C8
:100FD000E75E050EE7CFDBFF02D0050EDB6A040EED
:100FE000DBCF14F0160E45D9D880145414E2160E37
:100FF000DBCFE6FF150EDBCFE6FF040EDBCFE6FF0F
:10100000050EDB50E552E75CE552D880E754E55227
:10101000D880E7545FD9030EDB50010B0BE1080EBB
:10102000DB5008E0B2D801E08DD0080EDB50BED80E
:10103000080EDB6A170EDB5007E088D9170EF1D9CE
:1010400003E1151C01E17ED0160EDB5016E07ED9BF
:10105000300EE66E9FD802E1151C74E077D9DFCF21
:10106000E6FFC3EC0DF0E552E552E552F4CF15F082
:101070000001F31C02E1151C65E0050EDBCF14F046
:10108000160EDB50D880145409E2050EDBCFE7FFC3
:10109000160EDB50E75E050EE7CFDBFF300EE66E87
:1010A000050ECBD94FE1390EDB2ADBCFE9FF3A0E33
:1010B00001E3DB2ADBCFEAFF090EEFCFDBFFDB50DA
:1010C0000EE044D9090EADD902E1151C3BE0390E02
:1010D000DB2ADBCFE9FF3A0EEDE3DB2AEBD755D86D
:1010E00031E1160EDBCFE6FF080EC3D8E552E72448
:1010F0005DD82ED0070EDB50030A1CE0010A14E075
:10110000030A07E07BD9DBCFEEFF020EDBCFEDFF5A
:101110001FD0F5D8196A17AE02D0186819682CD8F4
:10112000BCD819C0EEFF14D0EAD817BE186824D86E
:10113000B4D80ED063D9DBCFEFFF0AD07BD905E15D
:10114000151C03E1F368F46810D0FCD801E3DB2A36
:1011500079D947EF04F0010EDBCF14F0020EDBCF9C
:1011600015F014C0F3FF15C0F4FF3B0EE15C02E282
:10117000E16AE552E16ECBD029D9020EADEF09F05C
:1011800061D90800F550DF6E1200200EE66E080EE1
:101190001DEF0AF0C3EC0DF0E552E552E552F3CF36
:1011A00014F0F4CF15F00001F31C1200146E156A50
:1011B000D950010F4DD91450EE261550ED221200D2
:1011C000185E000E195AF70E18C0DBFFF80E19C092
:1011D000DBFF18C0E9FF19C0EAFF1200DBCFF4FF04
:1011E000F350F45C1200DB50E76E040EE7CFDBFF38
:1011F00012000A0EDBCF14F00B0EDBCF15F00C0E35
:10120000DBCF16F00D0EDBCF17F0145015101610B3
:1012100017101200130EEECFDBFF140EEDCFDBFF25
:10122000130EDBCF14F0140EDBCF15F00001800E8F
:1012300015141200F70EDBCF18F0F80EDBCF19F003
:101240001200050EDB50E66ED950130F01D9E5529E
:10125000E750EE6EED6A12000A0EDBCF06F00B0EC1
:10126000DBCF07F00C0EDBCF08F00D0EDBCF09F063
:101270001200DBCFE6FF150EDBCFE6FF050EDB50DD
:10128000E552E724E552E7241200DB50CED8010EE8
:10129000F36E060EF3CFDBFF1200EE50EFCFEAFF46
:1012A000E96E16C0EEFF17C0EEFF18C0EEFF120089
:1012B000D9CFE6FFDACFE6FFE1CFD9FFE2CFDAFF01
:1012C0001200DFCFE6FFE66AC1EC0EF0E552E55210
:1012D000F3501200E76E080EE7CFDBFF1200EECFEF
:1012E00014F0EECF15F0EFCF16F0176A1200050ECE
:1012F000DBCF14F0150EDB50D88014541200010E11
:10130000DBCF16F0020EDBCF17F0186A1200E552A1
:10131000E5CFDAFFE7CFD9FF12000A0E14C0DBFFDA
:101320000B0E15C0DBFF1200D9500A0F28EF0AF090
:10133000F36E070EF3CFDBFF1200EECF14F0EFCF0A
:1013400015F01200010EDB2A020E1200FC0EDBCF9C
:10135000E6FFFD0EDBCFE6FF1200145E000E155A0D
:10136000F70E14C0DBFFF80E15C0DBFF14C0E9FF59
:1013700015C0EAFF1200DA20EA6EEF2AEECFF6FF80
:10138000000EEF22EECFF7FFEF22EECFF8FF1200B4
:10139000040EDBCFE6FF130EDB50E552E75C9ADF6D
:1013A000DB5004DF060EDB501200090EDB500A0D85
:1013B000F350DF24D00FE76E090EE7CFDBFFC0EF5D
:1013C00008F0DB50F36E050EEEEF08F0F70EDBCF02
:1013D00014F0F80EDBCF15F01200DFCFE6FFCAEFF6
:1013E00008F028DF030EECDE6FEF09F01CEC04F0D0
:1013F000E552E552E552E55200091200BDDEEE501D
:10140000EFCFEAFFE96E010E1200130EDB50F36E10
:10141000040EEEEF08F0040EDB50F36E090EEEEF53
:1014200008F0DBCFE6FFCAEF08F0E76E050EE7CF66
:10143000DBFF12008BDFEDEF09F0DBCFE6FF86DF8D
:10144000F6EF09F0D950F90FE96EFF0EBBEF09F086
:0A145000E96E000EDA20EA6E1200C9
:06145A00D9CFE6FFE1CF4F
:10146000D9FF040EE126DE6ADE6ADE6ADD6ADD523D
:10147000DD52FD0EDBCF14F0FE0EDBCF15F0166A49
:10148000176A15AE02D016681768D9CFE9FFDACF10
:10149000EAFF030EEB501718E8AE02D0173408D05D
:1014A0001450EE5C1550EE581650EE581750EE588A
:1014B0000FE20C0EE66ED3EC0EF0E552D9CFE9FF49
:1014C000DACFEAFFEE2A000EEE22EE22EE22D1D78C
:1014D000040EE15C02E2E16AE552E16EE552E7CF1B
:1014E000D9FF12000F0EC16E070EB46E936A300E54
:1014F000926E0F0E946EF19E816A80901200D9CF89
:10150000E6FFE1CFD9FF020EE1268250020B01E097
:10151000010E080DF3CF16F08250010B040DF3CF2E
:1015200015F08050200B01E0010EE824146E80506D
:10153000100B01E0010E142415241624DE6EDD6A62
:10154000DECF14F0DDCF15F014C0F3FF15C0F4FFAB
:10155000020EE15C03E200D0E16AE552E16EE55281
:10156000E7CFD9FF12008092320EE66E0FEC0FF03B
:10157000E5528084320EE66E0FEC0FF0E552809457
:10158000320EE66E0FEC0FF0E55212008082320E42
:10159000E66E0FEC0FF0E5528084320EE66E0FEC33
:1015A0000FF0E5528094320EE66E0FEC0FF0E5522C
:1015B0001200380E816ED7DF320EE66EE66A4DDF1E
:1015C000E552E552010E816ECEDF320EE66EE66A1E
:1015D00044DFE552E5520D0E816EC5DF320EE66E38
:1015E000E66A3BDFE552E552060E816EBCDF320E45
:1015F000E66EE66A32DFE552E5521200010E816EB8
:10160000B2DF0A0EE66EE66A28DFE552E552120006
:10161000D9CFE6FFE1CFD9FF020E816EA4DF0A0E1B
:10162000E66EE66A1ADFE552E552FD0EDBCFE6FF15
:10163000FE0EDB50280DF350E552E724E76EFE0E58
:10164000E7CFDBFFFD0EDB6AFE0EDB50F36EFD0E17
:10165000DBCFF4FFF350F45C0BE2140E816E83DFFA
:10166000320EE66E0FEC0FF0E552FD0EDB2AECD7E2
:10167000E552E7CFD9FF1200D9CFE6FFE1CFD9FF7E
:10168000FE0EDB50816E82DF320EE66E0FEC0FF045
:10169000E552E552E7CFD9FF1200D9CFE6FFE1CFFF
:1016A000D9FFFD0EDBCFE9FFFE0EDBCFEAFFEF50E7
:1016B0000EE0FD0EDBCFE9FFDB2AFE0EDBCFEAFFFB
:1016C00001E3DB2AEF50E66ED7DFE552EAD7E552B9
:1016D000E7CFD9FF12000201246B300E926EF00E9C
:1016E000936EEF0E206F20C281FF040E216F2151F7
:1016F000000821E22051FE0BE842206F20C281FF4A
:10170000050EE66EE66AA9DEE552E5528150100B41
:1017100009E08150200B06E08150400B03E081502E
:10172000800B01E10AD80201240502E1255104D011
:101730002105216FDCD7CFD71200F00E936E81CF39
:1017400023F202012315226F0F0E2015206F205166
:101750002211206F81CF23F2F00E2315226FF00E9D
:10176000225D01E0F7D7936A06D826C225F202016E
:10177000010E246F12000201276B100E275D14E288
:101780002751EA6A000FE96E020EEA22EF50205D4F
:1017900008E12751EA6A100FE96E020EEA22EFCF44
:1017A00026F22729276FE9D726C281FF640EE66E4D
:1017B000E66A53DEE552E55212000201286B070E7D
:1017C000285D1DE288DF0201296F2851EA6A2A0F8D
:1017D000E96E020EEA2229C2EFFF2851EA6A2A0FB7
:1017E000E96E020EEA22EF50460802E108D004D06A
:1017F00029C2E6FF41DFE5520201282BE0D728513C
:10180000EA6A2A0FE96E020EEA22EF6A120002016A
:10181000286B070E285D16E22851EA6A2A0FE96E46
:10182000020EEA22EF50E66E27DFE5520201282978
:10183000EA6A2A0FE96E020EEA22EF5001E102D0B5
:10184000282BE7D71200D9CFE6FFE1CFD9FFE65228
:10185000F250800B01E0010EDF6EF29EA69EA69C68
:10186000A684FE0EDB50A96EFD0EDB50A86E550E51
:10187000A76EAA0EA76EA682A6B2FED7A694DF50C8
:10188000E8B0F28EE8A0F29EE552E552E7CFD9FF2C
:101890001200D9CFE6FFE1CFD9FFA69CA69EFE0E8F
:1018A000DB50A96EA680A85000D0E552E7CFD9FF43
:1018B000120018DE7EDEA2DE2A0EE66EDDDEE552C6
:1018C0007CDF2A0EE66E020EE66EA9EC0CF0E55205
:1018D000E552F3CF33F2F4CF34F290DE2A0EE66E07
:1018E000CBDEE5526ADF2A0EE66E020EE66EA9EC4A
:1018F0000CF0E552E552F3CF35F2F4CF36F20201A7
:1019000033513525376F34513621386F77DE37C282
:10191000E6FF38C2E6FF450E146E1E0E156E166AFF
:1019200014C0E6FF15C0E6FF16C0E6FF390EE66EEE
:10193000020EE66E1EEC0DF0176E070EE15E1750FC
:10194000390EE66E020EE66EA8DEE552E552FFD7CE
:02195000120083
:0E195200FF0EE3CFEAFFE552FF0EE3CFE9FF01
:10196000E552E66AE66AD9CFE6FFDACFE6FFFC0E7B
:10197000E124D96EFF0EE220DA6EE66AE66AE66AD4
:10198000200EEF5C06E0090EEF5C03E0EF6603D08B
:101990003FD0EE50F5D72D0EEF5C03E1FF0EE32AAA
:1019A00003D02B0EEF5C01E1EE502F0EEF6424D03C
:1019B0003A0EEF6021D0D890F90EE336FA0EE336F6
:1019C000FD0EDECFE3FFFE0EDDCFE3FFD890F90E74
:1019D000E336FA0EE336D890F90EE336FA0EE33624
:1019E000FD0EE350DE26FE0EE350DD22300EEE5CEF
:1019F000DE26000EDD22D9D7FF0EE3CFE8FFE85246
:101A000007E0F90EE31EE32AFA0ED8B4E306E31E5C
:101A1000E552E552E552FF0EE3CFDAFFE552FF0E45
:101A2000E3CFD9FFE552E1CFE9FFE2CFEAFFED5284
:0C1A3000ED52EECFF3FFEFCFF4FF1200F9
:041A3C00D9CFE6FF19
:101A4000DACFE6FFE1CFD9FFE2CFDAFFE652E65286
:101A5000E652E652D950F90F146EFF0EDA20156ED9
:101A6000020E14C0DBFF030E15C0DBFF020EDBCF3E
:101A7000E6FF030EDBCFE6FFF90EDBCFE6FFFA0E43
:101A8000DBCFE6FFFB0EDBCFE6FFD950FC0FE66EA7
:101A9000FF0EDA20E66E32EC04F0146E070EE15C05
:101AA00002E2E16AE552E16E1450F3CFDEFFF4CFBB
:101AB000DDFFFC0EDBCFE9FFFD0EDBCFEAFFEF6AB7
:101AC000DECF14F0DDCF15F014C0F3FF15C0F4FF26
:101AD000040EE15C02E2E16AE552E16EE552E5CF17
:081AE000DAFFE7CFD9FF120085
:081AE8002A0EF66E080EF76EDF
:101AF000000EF86E00010900F550656F0900F55001
:101B0000666F03E1656701D03DD00900F550606F55
:101B10000900F550616F0900F550626F0900090076
:101B2000F550E96E0900F550EA6E09000900090058
:101B3000F550636F0900F550646F09000900F6CF96
:101B400067F0F7CF68F0F8CF69F060C0F6FF61C0CA
:101B5000F7FF62C0F8FF0001635302E1645307E03E
:101B60000900F550EE6E6307F8E26407F9D767C025
:101B7000F6FF68C0F7FF69C0F8FF00016507000EB7
:061B8000665BBFD71200F6
:0A1B8600D9CFE6FFDACFE6FFE1CF8A
:101B9000D9FFE2CFDAFFFB0EDBCF14F0FC0EDBCF78
:101BA00015F00001800E15141AE1FB0EDBCFE9FFE2
:101BB000FC0EDBCFEAFFEECFF3FFEDCFF4FFEE2A12
:101BC000000EEF22F3CFE9FFF4CFEAFFFD0EDBCFEB
:101BD000EFFFEF50156AF36E15C0F4FF10D0FB0E47
:101BE000DB50FE0806E1FD0EDBCFE6FF01EC0FF057
:101BF00005D0FD0EDBCFE6FF24EC0FF0E552E552F9
:0A1C0000E5CFDAFFE7CFD9FF1200AD
:061C0A0006500B02F3CFAF
:101C100002F0F4CF03F00C02F3500326000EF42080
:101C2000046E06500D02F3500426000EF420056EDB
:101C300006500E02F350052607500B02F350032600
:101C4000F4500422000E052207500C02F350042623
:101C5000F450052207500D02F350052608500B02E0
:101C6000F3500426F450052208500C02F3500526C8
:0A1C700009500B02F3500526120084
:061C7A00FE0EE3CFE9FFBE
:101C8000FF0EE3CFEAFFF36AF46AEE5203E0F34A91
:101C9000F42AFBD71200FF0EE3CFF8FFE552FF0E48
:101CA000E3CFF7FFE552FF0EE3CFF6FFE552E66A1A
:101CB000E66AE66A0900F55209E0FD0EE32A05E14D
:101CC000FE0EE32A02E1FF0EE32AF4D7FD0EE3CF76
:101CD00007F0FE0EE3CF08F0FF0EE3CF09F012008D
:101CE00009C013F008C012F008500D02F4CF07F03D
:101CF000F3CF06F009500E02F4CF09F0F3CF08F04D
:101D00000D02F3500726F4500822E86A0922125007
:101D10000E02F3500726F4500822E86A09220EAE9C
:101D200096EF0EF01250085E1350095A13AE000CD5
:0A1D30000D50085E0E50095A000C19
:061D3A00056A046A036A59
:101D4000026A200EE76ED890063607360836093646
:101D500002360336043605360B50025C0C5003582D
:101D60000D5004580E50055809E30B50025E0C50FC
:101D7000035A0D50045A0E50055A062AE72EE4D78E
:021D800012004F
:0E1D8200F36AF46AFF0EE124E96EFF0EE22020
:101D9000EA6EED6607D02F0EEF6404D03A0EEF60C6
:061DA00001D0F32A12003D
:0A1DA600FF0EE3501B6E480E01D043
:101DB0004C0EE76EE72EFED7E76AE72EFED71B2E06
:061DC000F7D7000012003D
:0A1DC600000EF36E00EE00F0080EB0
:101DD00001D81200EA6002D0EE6AFCD7F350E96045
:061DE0001200EE6AFCD7C0
:0A1DE60012EE40F022EE40F0F86A21
:101DF000019C74EC0DF025EC0FF059EC0CF0FBD7C6
:021E00001200CE
:0E1E0200FF0EE350ACBA04D0AF6AAB8EAC8AD0
:0E1E1000949CACA2FED7AD6EF36EF46A120085
:021E1E00FF0EB5
:101E2000E350E84E1200000000D000D000D0E82EB1
:041E3000FAD71200CB
:0C1E3400303132333435363738396162D2
:051E400063646566000B
:031E450025640011
:021E4800120086
:021E4A00120084
:041E4C00EEEDEBE7E5
:101E5000DEDDDBD7BEBDBBB77E7D7B773031323375
:0C1E60003435363738394142434445469A
:00000001FF
